:020000040000FA
:06000000FE300F306A28FB
:08000800A000030EA100831209
:10001000C31D3B288B1C34288B1031181628B11CAB
:10002000342864300102031833281A2800001828E5
:1000300019281A281B281C281D281E281F2820289C
:1000400021283110B114A810031005190314AA0DAA
:10005000A90DA80DB00B342831152A08AF002908C6
:10006000AE002808AD00B11081010B11210E8300F4
:10007000A00E200E090005194328831601178312CC
:10008000B23081005E2883160113831203140B190A
:100090000310A80DA90DAA0DAB0DAC0DAC16FF30C9
:1000A0002C02031D5E28FA302B02031D5E28311539
:1000B0002A08AF002908AE002808AD008B100B11EC
:0A00C000210E8300A00E200E09009F
:0400CA0000340034CA
:0C00D400203084008001840A8030040287
:1000E000031C6C281230B0005A30C000C10001302F
:1000F000D400D500E400E500E300F100F000EE00DC
:10010000CC000730D8008030D7001F30E60007173A
:10011000FA30FD000A30EF008B13903003178D008A
:1001200083168C130C1483120C080313C7008B174F
:1001300083160F308505203086050D308705831224
:10014000850186018701103083168E00831270307E
:1001500083168F00831200300317990003130030B9
:1001600003179A0003130030970000309F000030FF
:1001700083169F008312003003179E000313003084
:1001800003179F000313C0308316810083123130A0
:1001900090000030920000308316940083120030EB
:1001A0009400A630831698008312003083169B00BB
:1001B00083129030980033308316990083120030F8
:1001C00083168C008312003083168D00831210304A
:1001D0008B000D16032681018E018F010B118B10F0
:1001E0000B108C128C018D010D168B174A23952351
:1001F0009A21E6170230C800382131194F24311AEC
:100200005221591C2D235918BE2200238F0803198F
:10021000FC288F01CB2331220322B121DA211729B7
:10022000E71BEB01EB0B1729E801E901EA01E713F2
:100230005918FC28B1192D29D60BFC28B11A0A30FF
:10024000B11EC830D600B11A34299A210310CC0D42
:10025000CC1E2D294A140830CC00B111B11A0A3035
:10026000B11EC830D600FC289A21BE180326FC28EF
:100270006400C31DB113C31D0800311808000B1D15
:1002800008000B11B11031141230B000051D4D29BA
:10029000B1178316011383120800B11383160117D7
:1002A00083120800311221305B02031D5D295C08B6
:1002B000CE005D08CF00661786295B085C065D02EC
:1002C000031D080077305B02031D6A295C08740671
:1002D000C400862966305B02031D71295C08CB00CF
:1002E000862955305B02031D78295C08F8008629B1
:1002F00044305B02031D7F295C08FA0086293330F5
:100300005B02031D8E295C08FB0086290310CC0CC0
:10031000031C95294A100130CC0095290310CC0DFF
:10032000CC1E95294A140830CC00B116B1110A3000
:10033000D6000800591459158B138316071283121F
:100340008B17071608005910D9101930DE00B112AA
:10035000B111C830D6008B138316071683128B1782
:1003600008000518B8291930C0070318BD2908006E
:100370000A30C002031CCF290800FF30C00042141D
:1003800064304102031808004210C2144317C3141A
:10039000F51BC3107717E6172830C8000800C00106
:1003A0004210C213C21C0800C2014313E6172C30CE
:1003B000C80008008518E1291930C1070318E6298B
:1003C00008000A30C102031CF8290800FF30C100F0
:1003D00042146430400203180800421042154317CB
:1003E000C310F51BC3147717E6172A30C80008009E
:1003F000C1014210C213421D0800C2014313E61797
:100400002E30C8000800E303031D0800E0080319AC
:10041000162A65186008E5186108651962089900D0
:100420000330E3000310E50DE51D08001430E30080
:100430000130E500EE080319282AEE030319262AE5
:100440006030E605031D282AE00108001F30E6049D
:100450000310E40D03186414640866050319282AC0
:100460004A2B8C1E0800E7174A150717FA30FD00C3
:100470001819CA146908E8006A08E9001A08EA00AD
:10048000E81F08006808C13C031D4E2A69086A0578
:10049000C3046A096904C3055725BD2A6808C23C1C
:1004A000031D5A2A69086A05C5046A096904C50555
:1004B0005D25BD2A6808C43C031D612A6908F70050
:1004C000BD2A6808FC39E03C031D722A69086818D7
:1004D0008038BB006A08E8188038BA00D625BE14F8
:1004E0003E14BD2A6808FC39F03C031D932A6908B4
:1004F00068188038EC008B136C0803178D00831686
:100500008C130C1483120C080313ED008B176C086A
:1005100000300319ED006C0348300319ED00323050
:10052000EE00E616BD2A6808FC39803C031DA22AAD
:10053000690868188038CE006A08E8188038CF004B
:10054000D815BD2A6808FC39903C031DAD2A6908FE
:1005500068188038CE005816BD2A6808A03C031DD4
:10056000BD2A69086A188038CD00C310EA18C31480
:1005700045126A194516D816BD2A08005919CB2A02
:10058000D3030F305305031D0800D3080319CE2AE7
:100590000716D30E0800591BA1235913071259112E
:1005A000D918A32955185008D518510855195208BB
:1005B0005705031DDE2AFF30D300E12A2230D30085
:1005C000E12A0310D70C0318E62A08008030D70070
:1005D0000310D50DD519ED2A08000130D5000430DF
:1005E000D819D4000830581AD4000310D40D0318B9
:1005F0005414540858050319ED2A9523D9140800FA
:10060000EF0B08000A30EF00061E2B2B0516031017
:10061000F00D031C192B0130F0000310F10D711EB9
:10062000192B0130F100F0004408F300C31BF3174D
:10063000051271187308F118720871197708F11D05
:10064000242B4B084A1880387005061203198516AA
:10065000031D8512080006160800DA0A0319D916C8
:100660005916071E5912D91D462B591A462BB1157A
:100670005A08283CD91A0310DD0DDC0DDB0DDA0118
:10068000D912DE0B462B31161930DE00D915591E52
:10069000D9110800E001E101E201E41F562B4F30BF
:1006A000E0004808E1004908E200E613641F5F2B00
:1006B0004830E0004E08E1004F08E2006613E41EF7
:1006C000682B4730E0006C08E1006D08E200E6129C
:1006D000641E742B4130E000390884000008E100FA
:1006E0003D0884000008E200E41D7C2B4C30E00053
:1006F0007708E1007808E200641D842B4530E000B3
:100700004A08E1004B08E200E41C8C2B4630E00074
:100710004308E1004408E200641C942B5830E000D8
:100720005930E1005A30E2000800D001D101D20175
:10073000541C9F2BF730D0004308D100C72BD41C8A
:10074000A62BA130D0007708D100C72B541DAD2BAC
:10075000A230D0004508D100C72BD41DB72BC13023
:10076000D0004E08D1004F08D200D8110800541E06
:10077000BF2BC230D0004E08D1005812C72BD41E58
:100780000800A730D0004D08D100D812C72B500860
:100790005106D2000800311FD02BFC03031931137E
:1007A000451BD72B071FD72BFD0303190713C70BB7
:1007B000FB2B8B13903003178D0083168C130C14B6
:1007C00083120C080313C7008B170310B20D0F30F0
:1007D0004418B200B21FF52BE6171E30C8003208CD
:1007E000C9004313321F4A16B201431BCA11431BEF
:1007F0004A12CB1B431307184311071C4315071953
:10080000C311071DC31587194312871D4316751C95
:100810000D2CC31E0D2C87140E2C8710FE0B080008
:1008200044188926441C8712770878020319871612
:10083000451F1F2C8526071F8716071B87124A1C7A
:1008400087174A188126790AF71BF707771B2C2C84
:10085000790A77020318F7007808F2000310790C80
:10086000013E7802C3130318F2000318C317C31222
:100870000310790C013E460778020318C316460898
:100880007802031CC3160310790C013E4602031CB8
:1008900008007802031CC3120800871408003111F5
:1008A000311B0800591808004A100717FA30FD00DC
:1008B000B7010430B8000C30370230300318B807E5
:1008C000C319B8178B1320303707380703178D006B
:1008D00083168C130C1483120C080313A400A500B8
:1008E000C030A50610303707380703178D00831670
:1008F0008C130C1483120C080313A300A6000230FF
:10090000A60600303707380703178D0083168C13AF
:100910000C1483120C080313A200A7000130A706D1
:100920008B17B11F992C22090339A200A309A4092E
:10093000A509C31DA82C22082D02031D512D230833
:100940002E02031D512D24082F02031D052DB42C4A
:1009500024082F02031D512D23082E02031D052DEF
:1009600022082D02031D512DE6170A30C800370852
:10097000C90000303702031DC22C4318080043147D
:100980005725080001303702031DD92CFF30FC0029
:100990003117441CC314441CB9257519D32C4418B1
:1009A00043134418CA15441C43170130431BB200BB
:1009B000080002303702031DEA2CFF30FC0031171B
:1009C000441CC314441CC125441C43170130431B61
:1009D000B200080003303702031DF12C441CC3147D
:1009E00008003030370738077F3903178D0083162A
:1009F0008C130C1483120C080313F7005917441CB2
:100A00006325FF30FC003117512DC31D0C2D250827
:100A10002F02031D512D142D26082E02031D512DCA
:100A200027082D02031D512DE6170C30C80037088A
:100A3000C90000303702031D222D431C080043105B
:100A40005725080001303702031D392DFF30FC0007
:100A50003117441CC310441CB0257519332D44189C
:100A600043134418CA15441C43170130431BB200FA
:100A7000080002303702031D4A2DFF30FC003117F9
:100A8000441CC310441CC125441C43170130431BA4
:100A9000B200080003303702031D512D441CC3105F
:100AA0000800B70A1C30370203180800592C2130FF
:100AB000BB004308BA00D62508002330BB00450818
:100AC000BA00D6250800771B0800431AAE2D031084
:100AD000790C013E77020318F7000318672D770899
:100AE00078020319852D03187D2D78087702C31825
:100AF0007902C318013EFF008C2D77087802C31CD1
:100B00007902C31C013EFF008C2D0310790C013EBD
:100B1000FF00F518F7079F2D0310790C013EF5181B
:100B2000013E7F02031C9F2D0310790C013EF70745
:100B3000790A77020318F7000318982D9F2D77087C
:100B400078024313031D4317E617C9003230C8006B
:100B5000F51843170130431BB20008009F2D080011
:100B60005917C310780AF700790A77020318F700BB
:100B700008005917C3147803F700790AF71BF70721
:100B8000080059170310790C78077902031CD02D3F
:100B90000319D02D0310790C013E7807F7000800E7
:100BA0000310790C013E7802F7000800FF010530C0
:100BB000DF000D123B08831203178D00831203130D
:100BC0003A08831203178C00831603178C130C1535
:100BD0008B138B1BE82D55308D00AA308D008C14A3
:100BE0008B170C11831203136400DF03031DFD2D0B
:100BF0000530DF00FF030319002E0D1EF42D080041
:100C00000C118B17D62D8B138B1B032E3130031732
:100C10008D0083168C130C1483120C080313F4003C
:100C20008B1774108B13323003178D0083168C13BF
:100C30000C1483120C080313F5008B178B1333303D
:100C400003178D0083168C130C1483120C080313E6
:100C5000F6008B173E18492E8B13213003178D0099
:100C600083168C130C1483120C080313C3008B1708
:100C700043138B13233003178D0083168C130C142E
:100C800083120C080313C5008B17C5124510C5103D
:100C900045138B13203003178D0083168C130C140F
:100CA00083120C080313C6008B17460A0319C601EA
:100CB0008B13303003178D0083168C130C148312A2
:100CC0000C08031307183030F900F9038B13803038
:100CD00003178D0083168C130C1483120C08031356
:100CE000B9008B178B13813003178D0083168C137B
:100CF0000C1483120C080313BD008B17BE103E109A
:100D000008000708803A870008000708403A870073
:100D100008000708203A87000800FF008926FF0B1B
:0C0D20008E2E08000708023A8700080029
:084000000F0000000000480061
:02400E00CC03E1
:1042000000004600FF00FF0040004200440046005E
:104210004200430040004100460047004400450082
:10422000FF00FF00FF00FF00F200F600FA00FE00B2
:10423000F000F200F400F600F800FA00FC00FE00C6
:104240000000FF00FF000000E500E500E500E500DC
:10425000E900E900E900E900E900E900E900E90016
:104260001800000001000000FF00FF00FF00FF0039
:104270000000010002000300040005000600070022
:104280004300420041004000470046004500440012
:104290004400450046004700400041004200430002
:1042A000F000F200F400F600F800FA00FC00FE0056
:1042B000F000F200F400F600F800FA00FC00FE0046
:1042C000ED00ED00ED00ED00ED00ED00ED00ED0086
:1042D000F100F100F100F100F100F100F100F10056
:1042E000080009000A000B000C000D000E000F0072
:1042F0001000110012001300140015001600170022
:104300007A007B00FF00FF000000000000000000BA
:104310000300030003000300030003000300030085
:10432000AA003000FF00FF00C800C800C800C80095
:10433000C800C800C800C800C800C800C800C8003D
:10434000FF00FF00FF00FF00C300F300CF00FF00ED
:104350000300C3003300F3000F00CF003F00FF0055
:10436000FF00FF00FF00FF00FF00FF00FF00FF0055
:10437000FF00FF00FF00FF00FF00FF00FF00FF0045
:10438000020002000200020002000200020002001D
:10439000000000000000000000000000000000001D
:1043A000C800C800C800C800C800C800C800C800CD
:1043B00088008800880088008800880088008800BD
:1043C0000300C3003300F3000F00CF003F00FF00E5
:1043D0000300C3003300F3000F00CF003F00FF00D5
:1043E000FF00FF00FF00FF00FF00FF00FF00FF00D5
:1043F000FF00FF00FF00FF00FF00FF00FF00FF00C5
:00000001FF
